:1000000063289200220884000930930003100D2019
:10001000920C930B072803140D2884139F1D1C2892
:10002000000820041F1D20068000841700082004FB
:10003000031C20068000272800082004031C20063B
:100040001F192006800084172009800527281F0D0E
:1000500006398C0030208D008C0A302000004A28A0
:1000600000308A000C0882070134753403341534DB
:1000700000343C340C34D9348F018E00FF308E07AD
:10008000031C8F07031C5E2803308D00DF304A20DD
:100090003E288D01E83E8C008D09FC30031C53285E
:1000A0008C07031850288C0764008D0F50280C18FB
:1000B00059288C1C5D2800005D2808008313031359
:1000C0008312640008008316FF308600013085002B
:1000D0008312A4010530A2000230A00004309F006A
:1000E000FF3001200B30012064000608803C031D16
:1000F00083280530A2000230A00004309F00FF30AA
:1001000001200130012064000608403C031D9228B4
:100110000530A2000230A00004309F00FF30012013
:100120000230012064000608203C031DA128053090
:10013000A2000230A00004309F00FF3001200330F5
:10014000012064000608103C031DB0280530A20001
:100150000230A00004309F00FF3001200430012055
:1001600064000608083C031DBF280530A2000230C9
:10017000A00004309F00FF30012005300120640002
:100180000608043C031DCE280530A2000230A00062
:1001900004309F00FF300120063001206400060873
:1001A000023C031DDD280530A2000230A00004300F
:1001B0009F00FF3001200730012064000608013C49
:1001C000031DEC280530A2000230A00004309F007F
:1001D000FF3001200830012064000608813C031D27
:1001E000FB280530A2000230A00004309F00FF3041
:1001F00001200930012064000608413C031D0A2942
:100200000530A2000230A00004309F00FF30012022
:100210000A30012064000608213C031D192905301D
:10022000A2000230A00004309F00FF3001200B30FC
:10023000012064000608113C031D28290530A20096
:100240000230A00004309F00FF3001200C3001205C
:1002500064000608093C031D2F291430A400640023
:100260000608053C031D3529A40164000608033C6B
:10027000031D44290530A2000230A00004309F0075
:0E028000FF3001200F30012024083C2074289C
:02400E00F53F7C
:00000001FF
